:020000040000FA
:0A0000000000000029EF00F039D0E5
:0800180076D09EA8FED7AD6E64
:100020001200096A086EFF0E0826092200D0D8A027
:100030001200030E076EE60E02D8F5D7076AFE0F10
:10004000066EE86A075AD8A012000000060600D023
:10005000F8D7006A4F0EAF6EB06A240EAC6E900EE9
:10006000AB6E00010F0EC16E070EB46EC69A470E3E
:10007000926EE00E936EC00E946E59D09EAA17D069
:10008000ABA404D0AE50AE50AB881100ABA205D0EB
:10009000AE50AE50AB98AB881100232A00EE25F08D
:1000A0002350E926000EEA22AECFEFFF1100F2A4A2
:1000B00009D0F294104A112AD6CF0EF0D7CF0FF004
:1000C000817A11002350245C0AE0242A00EE25F0F6
:1000D0002450E926000EEA22EF50226E01D0226859
:1000E0001200256A236A246A9D8A9F8AF28EF28C06
:1000F00012009D9A256A236A246AAE50AE50AB98CE
:10010000AB889D8A1200F29EE0CF26F3D8CF27F36A
:10011000E8CF28F3F28E0001A192F29E26C3E0FF01
:1001200027C3D8FF28C3E8FFF28E10001000CB6869
:10013000BE6A0C0EBD6E9494BB6ABA6E9492050EA4
:10014000CA6E7F0ECB6EBE6A0C0EBD6E9494BB6AF7
:10015000BA6E9492939A8A9ACF0EBD16000EBD1273
:10016000000EBE6ECF0EBA16000EBA12000EBB6E97
:100170001D6A939A8A8A320E54DF939A8A9AB1DF63
:10018000B8DFCD6AF294F28A870ED56EB16AA19279
:10019000A082D08EA292B00EB16E3AD90301256929
:1001A0001B503BDF420E39DF400E37DF0001D6CF58
:1001B0000EF0D7CF0FF086DF22C012F0BC0E125C1B
:1001C00007E3FE0E125C02E3F9D002D0146AF6D007
:1001D00012AE21D0146A8B0E125C05E112C014F02D
:1001E0001568166817D09B0E125C05E112C014F05A
:1001F000176818680FD0AB0E125C05E112C014F03E
:1002000019681A6807D0BB0E125C04E112C014F022
:100210001B681C68D3D0145202E1D0D0CFD08B0E13
:10022000145C1DE1152803E112C015F016D012C0B0
:1002300016F0490E155C07E1CF0EBA16000EBA1281
:10024000000EBB6E09D04A0E155C06E1CF0EBD163E
:10025000000EBD12000EBE6E1568B0D0AFD09B0E62
:10026000145CD8A45AD0172803E112C017F053D059
:1002700012C018F0185215E1490E175C07E1CF0EB5
:10028000BA16000EBA12000EBB6E09D04A0E175CE9
:1002900006E1CF0EBD16000EBD12000EBE6E176831
:1002A0008DD01DA037D0490E175C19E101EE25F065
:1002B000D8901834E926000EEA22EECF02F0EFCFF4
:1002C00003F000EE02F0CF0EBA16EE38300BBA1281
:1002D000ED30F36EEF30BB6EF332BB321BD04A0E03
:1002E000175C18E102EE25F0D8901834E926000ECC
:1002F000EA22EECF02F0EFCF03F000EE02F0CF0ED5
:10030000BD16EE38300BBD12ED30F36EEF30BE6E21
:10031000F332BE32176852D051D0AB0E145CD8A461
:1003200041D0192803E112C019F03AD012C01AF0D6
:10033000490E195C19E101EE25F0D8901A34E9262E
:10034000000EEA22EECF02F0EFCF03F000EE02F053
:10035000CF0EBA16EE38300BBA12ED30F36EEF3026
:10036000BB6EF332BB321BD04A0E195C18E102EEB1
:1003700025F0D8901A34E926000EEA22EECF02F0DA
:10038000EFCF03F000EE02F0CF0EBD16EE38300BCB
:10039000BD12ED30F36EEF30BE6EF332BE3219682F
:1003A0000DD00CD0BB0E145C09E11B2803E112C078
:1003B0001BF003D012C01CF003D800D08170F6D619
:1003C000420E1B5C14E11C520FE11D90CF0EBA16B9
:1003D000000EBA12000EBB6ECF0EBD16000EBD127F
:1003E000000EBE6E1D6A02D01D801D680FD07B0EF0
:1003F0001B5C0CE1CF0EBA16000EBA12000EBB6EDB
:10040000CF0EBD16000EBD12000EBE6E1B68120090
:100410000101266B256B286BB40E276F020E136E3D
:100420000001800E135C1DE227C104F028C105F015
:100430001350020DF3CF0CF0F4CF0DF00C50042448
:10044000026E0D500520036E01EE25F0D890133496
:10045000E926000EEA2202C0EEFF03C0EFFF132AD6
:10046000DFE30201266B256B286B780E276F020EE7
:10047000136E0001800E135C1DE227C204F028C237
:1004800005F01350020DF3CF0CF0F4CF0DF00C502B
:100490000424026E0D500520036E02EE25F0D89064
:1004A0001334E926000EEA2202C0EEFF03C0EFFF7C
:0804B000132ADFE31200FFD75D
:020000040030CA
:0300010006170ED1
:020005008580F4
:060008000FC00FE00F40E5
:00000001FF
